:100000008C019D018F019001910192019301940156
:1000100095019601980199019A0183161030850087
:1000200000308600640027308100831294289B01F1
:100030000C089C006D200314980203182A2803144E
:100040000130990203182A28031401309A02031878
:100050002A281B149C031C086D2003149902031802
:100060003728031401309A02031837281B149C0305
:100070001C086D2003149A02031840280314412819
:100080001B0C00349B010C089C006D20031098078A
:10009000031C5528031001309907031C5528031031
:1000A00001309A07031C55281B149C031C086D2063
:1000B00003109907031C6228031001309A07031CE0
:1000C00062281B149C031C086D2003149A07031C50
:1000D0006B2803146C281B0C003482070034003496
:1000E0000A3400340034643400340334E834003417
:1000F0002734103401348634A0340F344234403471
:1001000082079834963480348207C034F934A4349A
:10011000B034993492348234F834803498347F3453
:1001200082070034B134BC34831600308600831259
:1001300011308C0009308D008E0106309D00172093
:100140000318A9288E0A8D03031D9F2803308C02F3
:10015000AC28422003308C0209308D0010301D077E
:100160009B009B031B0884000E088E0180009D03EA
:1001700001300C07031D9F2818088F0010088F00FE
:1001800011089000120891001308920014089300BF
:1001900015089400013095009701810100000000CE
:1001A0009D013C308C008B01103085008316183087
:1001B000850083120F301D078400000884209B00F7
:1001C000033003151D02031DE6289B131B08860040
:1001D0001D08000085000B1DF028970A0B11F3285D
:1001E00000000000000007309B009B0BF52800007A
:1001F0009D0A073003111D02031DDA280000033099
:100200009B009B0B012900009D018C0BDA2800004C
:1002100031309B009B0B0A29000000000B1D1329A5
:10022000970A0B111629000000000000FF3086001D
:100230001030850083161030850083120B19970A41
:100240000B110108990017089A009B019B0A85155C
:1002500085110B11010803111902031926299B0AA4
:100260009B099B0A1B0A98000310980D990D9A0D83
:100270000310980D990D9A0D0310980D990D9A0D74
:1002800003100030902093001A088F000130902056
:1002900094001908900002309020950018089100F1
:1002A00015080314910203185F290314013090020A
:1002B00003185F29031401308F0203185F29140803
:1002C0000314900203186929031401308F020318E4
:1002D000692913088F020F089A0010089900110865
:0802E0009800103085009428FD
:00000001FF
